:100000001CC036C035C034C033C032C031C030C06F
:100010002FC02EC02DC02CC02BC02AC029C028C084
:1000200027C026C025C026C128C12AC12CC12EC187
:1000300030C132C134C118C11AC111241FBECFE56D
:10004000D4E0DEBFCDBF12E0A0E6B0E0EEEDF7E019
:1000500002C005900D92A236B107D9F712E0A2E6D0
:10006000B2E001C01D92AE38B107E1F7CED2B5C300
:10007000C7CF80936B0295B380FF0DC09F7E81FF39
:100080000DC0977F82FF0DC09B7F83FD0DC0892F20
:10009000826085BB0895906181FDF3CF986082FDF9
:1000A000F3CF946083FFF3CF892F8D7F85BB0895B5
:1000B000882311F4AD9A0895AD9808951F93CF93B6
:1000C000DF9310E0C0E0D0E080E0D3DF219683E151
:1000D000C838D807C9F7C0E0D0E08FE0CADF219662
:1000E00083E1C838D807C9F71F5F143059F7DF918B
:1000F000CF911F9108955D9BFECF8CB90895DC01CF
:10010000EC91EE2359F080E05D9BFECFECB98F5F60
:10011000FD01E80FF11DE081EE23B1F70895382FBE
:100120006AE03BD33AD3292F832F64E636D36AE0C3
:1001300034D3992371F4222321F05D9BFECF205DFF
:100140002CB95D9BFECF832F6AE027D3905D9CB9CD
:1001500008955D9BFECF905D9CB95D9BFECF205DB9
:100160002CB9EFCF369A349BFECF85B10895982FE6
:1001700080E48FB9779BFECF9FB9779BFECF089520
:100180008230F1F1833088F0843009F445C0843046
:10019000E8F4939880E48FB9779BFECF6FB9779B93
:1001A000FECF939A609366020895882361F4C09805
:1001B00080E48FB9779BFECF6FB9779BFECFC09A53
:1001C000609363020895813079F008958530E9F7EE
:1001D000949880E48FB9779BFECF6FB9779BFECF61
:1001E000949A609368020895929880E48FB9779BFF
:1001F000FECF6FB9779BFECF929A60936402089509
:10020000979880E48FB9779BFECF6FB9779BFECF2D
:10021000979A609365020895C19880E48FB9779B9F
:10022000FECF6FB9779BFECFC19A609367020895A6
:100230000F931F9390E0FC013197EA30F10588F0AD
:1002400000E010E080E0602F9BDF81E0612F98DF0D
:1002500082E0602F95DF83E0612F92DF1F910F9185
:100260000895ED5EFF4F099407E016E0EBCF07E03D
:1002700017E0E8CF01E010E0E5CF01E011E0E2CFC8
:1002800002E011E0DFCF02E012E0DCCF04E012E098
:10029000D9CF04E014E0D6CF06E014E0D3CF06E0D7
:1002A00016E0D0CF90916202809161029817D8F544
:1002B000E0916202F0E0E259FD4F8081803398F1D5
:1002C000E0916202F0E0E259FD4F80818A3358F5F7
:1002D00020E03AE010C0E0916202F0E0E259FD4F08
:1002E00080818033F0F0E0916202F0E0E259FD4F4E
:1002F00080818A33B0F4239F802D1124E091620223
:10030000F0E0E259FD4F20812053280F80916202D6
:100310008F5F8093620290916202809161029817D0
:10032000D0F2822F089520E0FCCF809162028032CB
:1003300068F4E0916202F0E0E259FD4FE0818091C3
:1003400062028F5F809362028E2F0895E0E08E2F0D
:1003500008959091620280916102981740F4E091B3
:100360006202F0E0E259FD4F80818C3211F080E0B2
:100370000895809162028F5F8093620281E0089508
:1003800080916D02CCDE5D9BFECF8CE28CB98091BA
:100390006302C5DE5D9BFECF8CE28CB98091640266
:1003A000BEDE5D9BFECF8CE28CB980916502B7DE2C
:1003B0005D9BFECF8CE28CB980916602B0DE5D9BC6
:1003C000FECF8CE28CB980916702A9DE5D9BFECFE7
:1003D0008CE28CB980916802A2DE5D9BFECF8CE23C
:1003E0008CB980916B0281709ADE5D9BFECF8CE2AE
:1003F0008CB980916B0290E0827090709595879592
:100400008EDE5D9BFECF8CE28CB980916B0290E01A
:1004100084709070959587959595879580DE5D9B06
:10042000FECF8CE28CB980916B0290E08870907066
:1004300095958795959587959595879570DE5D9BA4
:10044000FECF8CE28CB980916A0269DE5D9BFECFA3
:100450008CE28CB980916C0262DE5D9BFECF8CE2F7
:100460008CB980E690E04BDE84E690E048DE0895AB
:10047000FF920F931F9380916102803228F4809144
:100480006102882369F47CDF80916A028823B9F4D1
:10049000AD9A80E2809361021F910F91FF900895C1
:1004A00010926202FFDE882391F0813031F18230B8
:1004B00061F18330D9F083E292E021DEE5CFAD989F
:1004C00080E2809361021F910F91FF90089541DFB8
:1004D000882341F0E7DE182F8630F0F082E890E0C4
:1004E0000EDED2CF87E690E00ADECECF32DF882361
:1004F000D1F486E092E003DEC7CF10926902109239
:100500006A028DEE90E0FBDDBFCF23DF882391F4FC
:1005100082EF90E0F4DDB8CF1CDF882399F481EB03
:1005200090E0EDDDB1CFBEDE80936C028DEE90E009
:10053000E6DDAACFB7DE182F8230A8F083E191E084
:10054000DEDDA2CFAFDE682F883020F087EC90E0B0
:10055000D6DD9ACF81E080936A02812F11DE8DEE85
:1005600090E0CDDD91CFF5DE882321F487E391E0A3
:10057000C6DD8ACF97DEF82E81E08F1520F488E55E
:1005800091E0BDDD81CFE5DE882321F48CE791E0A9
:10059000B6DD7ACF87DE082F823020F08DE991E03A
:1005A000AEDD72CFD6DE882321F481EC91E0A7DDA9
:1005B0006BCF78DE282F823020F082EE91E09FDD35
:1005C00063CF81E080936A028F2D90E081709070FC
:1005D000880F991F1170182B802F90E081709070F8
:1005E000880F991F880F991F182B822F90E0817018
:1005F0009070880F991F880F991F880F991F812B62
:1006000038DD8DEE90E07BDD3FCFFF920F931F939F
:10061000CF93DF938BE287BB87EC88BB8EEB84BBE9
:100620008EE785BB8EE981BB8CEF82BB80E287B908
:1006300088E886B910BC89E189B9599A88E18AB9F4
:1006400083E58DB981E08EB920B386B390E0807CDC
:10065000907095958795959587959595879595959E
:10066000879530E02076307035952795359527951C
:10067000359527953595279535952795822B809328
:100680006D0289E492E03BDD80916D0248DD80E5FA
:1006900092E035DD80E690E032DD8CE592E02FDD02
:1006A0000DDD80916A02882309F475C0AD988091B0
:1006B0006902BEDD80916902DCDCC0E0D0E000E0D0
:1006C00010E0E0E2FE2E80916A02882301F5369A5E
:1006D000349BFECF35B1809169028A3078F58091E4
:1006E0006902432F50E028E1829FC00111244B96FC
:1006F000841795071CF5832F68E14FD0809369021A
:100700008091690295DD80916902B3DC39DE5F99E1
:1007100027C02196C1F60F5F1F4F80916C0288237E
:1007200091F280916C0260916C02689FB00111247B
:10073000C8013FD0892B39F623DEC5CF80916902ED
:10074000882329F380916902432F50E028E1829F9A
:10075000C00111240397481759076CF25F9BD9CF4A
:100760009CB1943289F080916102803290F69A3285
:1007700071F080916102E82FF0E0E259FD4F908323
:100780008F5F80936102C5CF10926102C2CF70DE8D
:10079000F0926102BECFAD9A8ACF991B79E004C076
:1007A000991F961708F0961B881F7A95C9F78095B0
:1007B0000895AA1BBB1B51E107C0AA1FBB1FA617A8
:1007C000B70710F0A61BB70B881F991F5A95A9F7FA
:0E07D00080959095BC01CD010895F894FFCF5F
:1007DE00312E36000D0A006572726F723A206D6905
:1007EE007373696E6720616D706C69666965720DF1
:1007FE000A006572726F723A20616D706C6966697B
:10080E006572206D75737420626520302C20312C3A
:10081E0020322C20332C20342C206F7220350D0AE0
:10082E00006572726F723A206D697373696E67201C
:10083E006761696E0D0A006572726F723A206761A8
:10084E00696E206D757374206265206265747765BC
:10085E00656E203020616E6420370D0A006F6B0DBF
:10086E000A006572726F723A206D697373696E67F2
:10087E002076616C756520666F72204C4544203081
:10088E000D0A006572726F723A204C45442030207A
:10089E0076616C7565206D757374206265203020ED
:1008AE006F7220310D0A006572726F723A206D6997
:1008BE007373696E672076616C756520666F722042
:1008CE004C454420310D0A006572726F723A204C0D
:1008DE00454420312076616C7565206D75737420EA
:1008EE0062652030206F7220310D0A006572726FC2
:1008FE00723A206D697373696E672076616C7565E7
:10090E0020666F72204C454420320D0A00657272CB
:10091E006F723A204C454420322076616C7565200A
:10092E006D7573742062652030206F7220310D0A50
:10093E00006572726F723A206D697373696E67200B
:10094E0076616C756520666F72204C454420330DC0
:10095E000A006572726F723A204C4544203320763D
:10096E00616C7565206D7573742062652030206F23
:10097E007220310D0A006572726F723A206D6973C2
:10098E0073696E672074696D6520666163746F723A
:10099E000D0A006572726F723A20636F6D6D616E33
:1009AE0064206D75737420626520302C20312C20EC
:1009BE0032206F7220330D0A00426F617264200084
:1009CE002C204669726D7761726520000D0A0D0A42
:0209DE000020F7
:00000001FF
